:100000000C945E070C947B070C947B070C947B0785
:100010000C947B070C947B070C947B070C947B0758
:100020000C947B070C947B070C947B070C947B0748
:100030000C947B070C947B070C947B070C947B0738
:100040000C947B070C947B070C947B070C947B0728
:100050000C947B070C94A20C0C947B070C947B07EC
:100060000C947B070C947B07808183848687898A24
:100070008C8E8F9192949597989A9B9D9EA0A2A307
:10008000A5A6A7A9AAACADAFB0B2B3B5B6B7B9BA79
:10009000BCBDBEC0C1C2C4C5C6C8C9CACBCDCECF07
:1000A000D0D2D3D4D5D6D7D9DADBDCDDDEDFE0E1C0
:1000B000E2E3E4E5E6E7E8E9EAEAEBECEDEEEEEFB1
:1000C000F0F1F1F2F3F3F4F5F5F6F6F7F8F8F9F9E3
:1000D000FAFAFAFBFBFCFCFCFDFDFDFDFEFEFEFE5C
:1000E000FEFFFFFFFFFFFFFF0000891112239B327D
:1000F0002446AD573665BF74488CC19D5AAFD3BEF8
:100100006CCAE5DB7EE9F7F88110080193331A2207
:10011000A5562C47B7753E64C99C408DDBBF52AED7
:10012000EDDA64CBFFF976E802218B3010029913E7
:100130002667AF763444BD554AADC3BC588ED19FB7
:100140006EEBE7FA7CC8F5D983310A2091121803C7
:10015000A7772E66B5543C45CBBD42ACD99E508F97
:10016000EFFB66EAFDD874C904428D5316619F7097
:100170002004A9153227BB364CCEC5DF5EEDD7FC77
:100180006888E1997AABF3BA85520C4397711E6087
:10019000A1142805B3373A26CDDE44CFDFFD56EC57
:1001A000E9986089FBBB72AA06638F7214409D5167
:1001B0002225AB343006B9174EEFC7FE5CCCD5DD37
:1001C0006AA9E3B8788AF19B87730E6295501C4147
:1001D000A3352A24B1163807CFFF46EEDDDC54CD17
:1001E000EBB962A8F99A708B088481951AA793B627
:1001F0002CC2A5D33EE1B7F04008C919522BDB3A17
:10020000644EED5F766DFF7C899400859BB712A6E6
:10021000ADD224C3BFF136E0C1184809D33B5A2AF6
:10022000E55E6C4FF77D7E6C0AA583B418869197C6
:100230002EE3A7F23CC0B5D14229CB38500AD91BD6
:10024000666FEF7E744CFD5D8BB502A499961087A6
:10025000AFF326E2BDD034C1C3394A28D11A580BB6
:10026000E77F6E6EF55C7C4D0CC685D71EE597F476
:100270002880A1913AA3B3B2444ACD5B5669DF7896
:10028000600CE91D722FFB3E8DD604C79FF516E466
:10029000A9902081BBB332A2C55A4C4BD7795E6876
:1002A000E11C680DF33F7A2E0EE787F61CC495D546
:1002B0002AA1A3B03882B193466BCF7A5448DD5956
:1002C000622DEB3C700EF91F8FF706E69DD414C526
:1002D000ABB122A0B9923083C77B4E6AD5585C4936
:1002E000E33D6A2CF11E780F2D2D2D2D2D2D2D2D5A
:1002F0002D2D2D2D2D2D2D2D2D2D2D2D2D2D2D2D2E
:100300002D2D2D2D2D2D2D2D2D2D0A004820202079
:100310002020202020205072696E7420636F6E664A
:10032000696775726174696F6E0A0043202020202E
:100330002020202020436C65617220636F6E666907
:100340006775726174696F6E0A004C20202020204E
:10035000202020204C6F616420636F6E6669677592
:10036000726174696F6E0A005320202020202020C3
:1003700020205361766520636F6E666967757261D0
:1003800074696F6E0A00573C5858583E2020202050
:10039000536574207472616E736D697373696F6EE7
:1003A000207461696C2074696D6520696E206D73BD
:1003B0000A00773C5858583E20202020536574206E
:1003C000707265616D626C652074696D6520696E1F
:1003D000206D730A00563C312F303E2020202053E0
:1003E000696C656E74206D6F6465206F6E2F6F662B
:1003F000660A0A00763C312F303E202020205665C8
:1004000072626F7365206D6F6465206F6E2F6F660B
:10041000660A0070693C312F303E202020507269FE
:100420006E7420494E464F206F6E2F6F66660A0A23
:1004300000706D3C312F303E2020205072696E7468
:100440002044415441206F6E2F6F66660A00707021
:100450003C312F303E2020205072696E7420504174
:100460005448206F6E2F6F66660A0070643C312F0F
:10047000303E2020205072696E7420445354206F07
:100480006E2F6F66660A0070733C312F303E20205D
:10049000205072696E7420535243206F6E2F6F6626
:1004A000660A006D613C312F303E2020204175747A
:1004B0006F6D61746963206D657373616765204159
:1004C000434B206F6E2F6F66660A0A006D723C7395
:1004D0007369643E20205265747279206C61737474
:1004E000206D6573736167650A006D733C73736992
:1004F000643E2020536574206D65737361676520C9
:10050000726563697069656E7420535349440A00CB
:100510006D633C63616C6C3E2020536574206D6597
:10052000737361676520726563697069656E7420B5
:1005300063616C6C7369676E0A006C743C732F6145
:100540003E20202053656C6563742073796D626F63
:100550006C207461626C6520287374616E646172D2
:10056000642F616C7465726E617465290A0A006C8F
:10057000733C73796D3E20202053656C6563742055
:1005800073796D626F6C0A006C643C302D393E20CB
:10059000202053657420616E74656E6E61206469FD
:1005A00072656374697669747920696E666F0A0092
:1005B0006C673C302D393E20202053657420616EDD
:1005C00074656E6E61206761696E20696E666F0A80
:1005D000006C683C302D393E20202053657420612A
:1005E0006E74656E6E612068656967687420696EF7
:1005F000666F0A006C703C302D393E202020536518
:100600007420545820706F77657220696E666F0A87
:10061000006C6C6F3C4C4F4E3E2020536574206C38
:100620006174697475646520284E4D45412D666F6F
:10063000726D61742C2065672030373230312E376F
:100640003557290A006C6C613C4C41543E202053C4
:100650006574206C6174697475646520284E4D451D
:10066000412D666F726D61742C20656720343930BE
:10067000332E35304E290A0073323C737369643E61
:10068000202053657420504154483220535349442C
:100690000A0A0073313C737369643E202053657409
:1006A00020504154483120535349440A0073643C5C
:1006B000737369643E2020536574206465737469A4
:1006C0006E6174696F6E20535349440A0073633C32
:1006D000737369643E202053657420796F757220AE
:1006E000535349440A00323C63616C6C3E20202025
:1006F0005365742050415448322063616C6C7369B7
:10070000676E0A0A00313C63616C6C3E2020205306
:1007100065742050415448312063616C6C73696783
:100720006E0A00643C63616C6C3E2020205365744B
:100730002064657374696E6174696F6E2063616CA7
:100740006C7369676E0A00633C63616C6C3E2020C9
:100750002053657420796F75722063616C6C7369C6
:10076000676E0A00233C6D73673E2020202053658E
:100770006E642041505253206D6573736167650A42
:100780000A00403C636D743E2020202053656E6457
:10079000206C6F636174696F6E207570646174653D
:1007A0002028636D74203D206F7074696F6E616CDA
:1007B00020636F6D6D656E74290A00213C6461745D
:1007C000613E20202053656E642072617720706145
:1007D000636B65740A0053657269616C20636F6DA9
:1007E0006D616E64733A0A002D2D2D2D2D2D2D2D4A
:1007F0002D2D2D2D2D2D2D2D2D2D2D2D2D2D2D2D29
:100800002D2D2D2D2D2D2D2D2D2D0A0054582054FC
:1008100061696C3A20256C750A0054582050726545
:10082000616D626C653A20256C750A0053796D62C2
:100830006F6C3A2025630A0053796D626F6C2074E7
:1008400061626C653A207374616E646172640A005F
:1008500053796D626F6C207461626C653A20616CD3
:100860007465726E6174650A0044697265637469C7
:10087000766974793A2025640A004761696E3A20E6
:1008800025640A004865696768743A2025640A008F
:10089000506F7765723A2025640A004175746F2D98
:1008A00061636B206D657373616765733A204F6692
:1008B000660A004175746F2D61636B206D657373FB
:1008C000616765733A204F6E0A0050617468323A6E
:1008D00020252E36732D25640A0050617468313A44
:1008E00020252E36732D25640A0044657374696EC5
:1008F0006174696F6E3A20252E36732D25640A00C7
:1009000043616C6C7369676E3A20252E36732D2512
:10091000640A00436F6E66696775726174696F6E11
:100920003A0A00300A004572726F723A20496E76B8
:10093000616C696420636F6D6D616E640A0045725D
:10094000726F723A20496E76616C69642076616CD0
:10095000756520666F72205458207461696C0A00B6
:100960005458205461696C2073657420746F20257D
:100970006C756D730A004572726F723A20496E761B
:10098000616C69642076616C756520666F72207099
:100990007265616D626C650A00507265616D626CB2
:1009A000652073657420746F20256C756D730A0063
:1009B000310A004D657373616765206175746F2D31
:1009C00061636B2064697361626C65640A00310A5B
:1009D000004D657373616765206175746F2D616388
:1009E0006B20656E61626C65640A00310A005265B5
:1009F0007472696564206C617374206D65737361D2
:100A000067650A00310A000A002D25640A004D6559
:100A1000737361676520726563697069656E743AA6
:100A200020252E367300310A000A002D25640A00A5
:100A30004D65737361676520726563697069656E82
:100A4000743A20252E367300310A0053656C6563B5
:100A5000746564207374616E646172642073796D6F
:100A6000626F6C207461626C650A0053656C65632B
:100A700074656420616C7465726E6174652073794D
:100A80006D626F6C207461626C650A0053796D62EF
:100A90006F6C2073657420746F2025630A004469AD
:100AA0007265637469766974792073657420746FF4
:100AB0002025646465670A00446972656374697619
:100AC0006974792073657420746F206F6D6E690A84
:100AD00000310A00310A004761696E207365742095
:100AE000746F20256464420A00310A00416E746507
:100AF0006E6E612068656967687420736574207420
:100B00006F20256C646D204141540A00310A005069
:100B10006F7765722073657420746F202564770A7F
:100B200000310A004C6F6E677469747564652073D8
:100B3000657420746F20252E39730A00310A004C29
:100B4000617469747564652073657420746F202501
:100B50002E38730A0053696C656E74206D6F64657E
:100B60002064697361626C65640A0053696C656E28
:100B700074206D6F646520656E61626C65640A0047
:100B8000566572626F7365206D6F6465206469736A
:100B900061626C65640A00566572626F7365206DF0
:100BA0006F646520656E61626C65640A00310A00DD
:100BB0005072696E7420494E464F206469736162B9
:100BC0006C65640A00310A005072696E7420494EE7
:100BD000464F20656E61626C65640A00310A005000
:100BE00072696E7420444154412064697361626C7F
:100BF00065640A00310A005072696E7420444154E1
:100C00004120656E61626C65640A00310A005072B1
:100C1000696E7420504154482064697361626C6548
:100C2000640A00310A005072696E742050415448C1
:100C300020656E61626C65640A00310A0050726959
:100C40006E74204453542064697361626C65640A55
:100C500000310A005072696E742044535420656E4E
:100C600061626C65640A00310A005072696E74201A
:100C70005352432064697361626C65640A00310AEF
:100C8000005072696E742053524320656E61626C2D
:100C900065640A00310A0050617468323A20252EDA
:100CA00036732D25640A00310A0050617468313AA8
:100CB00020252E36732D25640A00310A0044657301
:100CC00074696E6174696F6E3A20252E36732D2516
:100CD000640A00310A0043616C6C7369676E3A20E4
:100CE000252E36732D25640A00310A005061746880
:100CF000323A20252E36732D25640A00310A005021
:100D0000617468313A20252E36732D25640A00312E
:100D10000A0044657374696E6174696F6E3A2025C8
:100D20002E36732D25640A00310A0043616C6C7302
:100D300069676E3A20252E36732D25640A00310A24
:100D4000004D6573736167652073656E740A0031C9
:100D50000A004C6F636174696F6E20757064617412
:100D6000652073656E740A00310A005061636B651B
:100D7000742073656E740A000D0A00444154413AB0
:100D800020005B252E36732D25645D2000504154D4
:100D9000483A20005B252E36732D25645D200044E3
:100DA00053543A20005B252E36732D25645D2000B8
:100DB0005352433A2000310A00436F6E66696775EB
:100DC000726174696F6E2073617665640A00300A1F
:100DD000004572726F723A204E6F2073746F7265A5
:100DE0006420636F6E66696775726174696F6E20E7
:100DF000746F206C6F6164210A00436F6E666967CF
:100E000075726174696F6E206C6F616465640A004D
:100E1000310A00436F6E66696775726174696F6E3F
:100E200020636C65617265642E2052657374617213
:100E30007420746F206C6F61642064656661756CEA
:100E400074732E0A002D2D2D2D2D2D2D2D2D2D2D94
:100E50002D2D2D2D0A004D6F64656D207265616426
:100E6000790A0044656661756C7420636F6E66690B
:100E70006775726174696F6E206C6F61646564215F
:100E80000A00756E7369676E65642E696F2F6D69F0
:100E900063726F617072730A004D6963726F4150C3
:100EA00052532076312E30620A002D2D2D2D2D2DFE
:100EB0002D2D2D2D2D2D2D2D2D0A000011241FBE81
:100EC000CFEFD8E0DEBFCDBF11E0A0E0B1E0EEECA7
:100ED000FDE402C005900D92A234B107D9F716E0E7
:100EE000A2E4B1E001C01D92A23CB107E1F70E946B
:100EF000D7200C94E5260C9400002FB7F89460914D
:100F0000B2047091B3048091B4049091B5042FBFE2
:100F100008950C941314789488EE93E00E94FD08D1
:100F200049E857E068EE73E084EC94E00E943B0DE2
:100F300086EB94E00E94B607ECEBF6E086EB94E0DB
:100F4000938382839183808384EC94E00C94A81231
:100F50009091C00095FFFCCF8093C60008958091CA
:100F6000C00087FFFCCF8091C6000895CF93DF9328
:100F7000CDB7DEB72E970FB6F894DEBF0FBECDBF4C
:100F8000DC018EE0FD01982F11929A95E9F71092FD
:100F9000C50097E69093C400E0ECF0E090819D7F5F
:100FA000908396E09093C20098E19093C1009E01D7
:100FB0002F5F3F4FF90111928A95E9F783E08C8307
:100FC00088EA97E09A8789878FEA97E09C878B87E2
:100FD0009EE0F90101900D929A95E1F72E960FB6D9
:100FE000F894DEBF0FBECDBFDF91CF910895811180
:100FF00006C08091C000881F8827881F089580E060
:1010000008958091C00087FF03C08091C6000895B5
:101010008FEF08950F931F93CF93DF93182FC091F5
:101020001A06D0911B06FE01E959FF4F80818111FC
:1010300024C080E490E09E8F8D8F1C8E1B8E1A8EB4
:1010400001E00083299A2091090130910A01409121
:101050000B0150910C01A0EBB4E00E944B216056B3
:10106000704F8F4F9F4F20E43FE140E050E00E94DF
:101070006A213B8B2A8B009393020FB7F89420913F
:101080000501309106014091070150910801A0EB44
:10109000B4E00E944B216056704F8F4F9F4F20E469
:1010A0003FE140E050E00E946A213D8B2C8B0FBF56
:1010B000E0911A06F0911B064FB7F89423A134A1D2
:1010C000878D90A12817390739F425A136A181A170
:1010D00092A12817390779F065A176A123A134A13F
:1010E0002150310991E080E06217730709F090E028
:1010F000292F382F02C021E030E04FBF232BC1F64B
:10110000E0911A06F0911B062FB7F894A5A1B6A19D
:101110001C9345A156A181A192A14817590719F422
:10112000878D90A103C085A196A1019696A385A362
:101130002FBFDF91CF911F910F910895E0911A0673
:10114000F0911B064FB7F894EB58FF4F248135817F
:10115000868197814FBF28173907E9F0E0911A0679
:10116000F0911B069FB7F894EB58FF4FA481B5810F
:1011700022813381A217B30719F42081318105C080
:10118000A481B5819D012F5F3F4F358324838C91CE
:101190009FBF90E008958FEF9FEF089581E08093C7
:1011A0009202089581E0809392021092800089E17A
:1011B0008093810081E896E0909387008093860079
:1011C00080919202882321F080E480937C0002C009
:1011D00010927C003898409880917E0081608093C6
:1011E0007E0087E080937B008CEE80937A008AB14A
:1011F000886F8AB9219A229A08950F931F93CF93EB
:10120000DF93CDB7DEB72E970FB6F894DEBF0FBED3
:10121000CDBF8C018AECD8011D928A95E9F7109315
:101220001B0600931A0680E490E0F801968F858FE4
:10123000C80180599F4FE859FF4F9183808397835E
:101240008683958384830496938382830996D80149
:10125000AB58BF4F11969C938E9317969C938E9389
:10126000169715969C938E931497CF9613969C93EE
:101270008E93129785599109D80190969C938E93DD
:101280005F9796969C938E93959794969C938E9346
:101290009397CF9692969C938E93919784E090E04B
:1012A000A681B7811C9246815781228133814217E2
:1012B000530719F42081318104C0268137812F5FC3
:1012C0003F4F37832683019759F70E94D2088EE05B
:1012D000FE013196DF01982F1D929A95E9F793E070
:1012E0009C832AE038E03A8729872EE938E03C875A
:1012F0002B87D80101900D928A95E1F72E960FB6B3
:10130000F894DEBF0FBECDBFDF91CF911F910F913B
:1013100008950F931F93CF93DF93E0911A06F091F6
:101320001B0625A136A134A323A3EC018C01060FD3
:10133000171FC017D10721F089910E940A08F9CF21
:10134000DF91CF911F910F910895DC0156968C91FA
:1013500056978111ECC058968C9158978111A2C074
:1013600093964D915C91949795962D913C9196977B
:101370004217530739F454962D913C915597232BDE
:1013800009F460C059969C915997911103C05A96DF
:101390001C925A9791E059969C93599752962D9189
:1013A0003C9153972115310599F593964D915C9198
:1013B000949795962D913C9196974217530759F41F
:1013C00054962D913C9155972150310955963C9357
:1013D0002E93549723C09396ED91FC9194979196F8
:1013E0002D913C919297E217F30729F45F962D9186
:1013F0003C91909707C09396ED91FC9194979F0133
:101400002F5F3F4F94963C932E939397908107C004
:101410002150310953963C932E9352979EE757964D
:101420009C93579757969C9157979B3189F5939624
:101430004D915C91949795962D913C91969742177A
:10144000530739F410929302A959BF4F1C9229985F
:1014500008959396ED91FC91949791968D919C911E
:101460009297E817F90729F45F968D919C919097D0
:1014700006C09396ED91FC919497CF0101969496B6
:101480009C938E939397808157968C93579706C021
:101490009E57923018F459961C92599781E05896AD
:1014A0008C93589759968C9159975D962D913C91B4
:1014B0005E978823A9F05A968C915A97853080F0D0
:1014C0005A961C925A972034310519F080E490E026
:1014D00002C085E790E05E969C938E935D9723C053
:1014E00058968C91589757969C915797982341F00E
:1014F0005A969C915A979F5F5A969C935A970FC001
:101500005A961C925A972034310519F020E430E0A5
:1015100002C025E730E05E963C932E935D97880FDE
:1015200058968C93589788E056968C9356975D966C
:10153000ED91FC915E975B968D919C915C97E80F85
:10154000F91F9F0131705C963C932E935B975696E2
:101550008C915697815056968C93FF27E038F10571
:1015600030F08FEF90E0AC014E1B5F0BFA01E859B1
:10157000FF4F84912F3F310511F008F080950895B9
:10158000EF92FF920F931F93CF93DF93FC018C0197
:1015900001541F4FD8014D915C91119712971196EC
:1015A0005C934E93A555B10914968D919C91159716
:1015B00012962D913C9113978217930721F42D9148
:1015C0003C91119707C014968D919C9115979C01A1
:1015D0002F5F3F4F15963C932E931497EC01288173
:1015E000260290011124C9019595879595958795B7
:1015F000E801998388837F01D3ECED0EF11CE701AC
:10160000288139818F010F531F4FE80139832883C7
:10161000840F951F35952795820F931FE7019983B6
:101620008883AF014B535F4F21E0181619060CF465
:1016300020E0EA018881880F822B888316968D919D
:101640009C911797EC01688316962D913C91179702
:1016500012968D919C9113972817390721F48D913B
:101660009C91119705C016968D919C9117970196A4
:1016700017969C938E931697DA019C91892F8695E5
:10168000869589278370DF01AA53BF4F833039F4D1
:101690008C91803214F48F5F01C081508C938C91B7
:1016A000885F803414F48C9346C18F738C93DF0170
:1016B000A953BF4F8C91880F97702BEF290F2330C0
:1016C00010F0933009F481608C938C91982F96954B
:1016D0008927809581709685990F892B86878E370B
:1016E00009F048C0DF01AB58BF4F14962D913C91D3
:1016F00015978D919C9111972817390761F41696CB
:101700002D913C91179712968D919C9113972817C4
:10171000390709F4DCC016962D913C911797149661
:101720008D919C91159701972817390709F4CFC01F
:101730001696CD91DC9117978EE7888316962D919A
:101740003C91179712968D919C9113972817390702
:1017500021F48D919C91119705C016968D919C91C5
:101760001797019617969C938E93169781E0818B1D
:101770002A9AB0C0982F9F779F3719F4118A2A9818
:10178000DAC09189992309F4D6C0982F9F739E33AC
:1017900009F4D1C080FF03C080898068808B978561
:1017A0009F5F97878089983008F499C0DF01AB5814
:1017B000BF4F92E8980F923018F08B3109F044C077
:1017C00014962D913C9115978D919C911197281706
:1017D000390759F416962D913C91179712968D91D1
:1017E0009C9113972817390759F116962D913C9122
:1017F000179714968D919C91159701972817390783
:10180000F9F01696CD91DC9117978BE188831696A7
:101810002D913C91179712968D919C9113972817B3
:10182000390721F48D919C91119705C016968D91E1
:101830009C911797019617969C938E93169704C0C8
:10184000118A2A9880E001C081E014964D915C9144
:1018500015972D913C9111974217530759F41696FD
:101860004D915C91179712962D913C9113974217C9
:10187000530769F116964D915C91179714962D9127
:101880003C911597215031094217530701F1908976
:101890001696CD91DC911797988316964D915C9191
:1018A000179712962D913C9113974217530721F4E5
:1018B0002D913C91119706C016962D913C9117974A
:1018C0002F5F3F4F17963C932E93169703C0118AB4
:1018D0002A9880E0108A1786882321F02CC08695EC
:1018E000808B29C0DF01A853BF4F8D919C91119728
:1018F000816011969C938E93EB58FF4F2481358124
:10190000808191812817390739F4268137818281B6
:1019100093812817390741F0268137818481958189
:1019200001972817390739F4868197819583848335
:1019300011961C921E92DF91CF911F910F91FF90F3
:10194000EF9008951F920F920FB60F9211242F93CC
:101950003F934F935F936F937F938F939F93AF9337
:10196000BF93EF93FF9380E286BB60917800709104
:1019700079007695679576956795605880911A06F7
:1019800090911B060E94C00A80919302882349F01F
:1019900080911A0690911B060E94A509807F88609D
:1019A00001C080E88BB98091B2049091B304A091FA
:1019B000B404B091B5040196A11DB11D8093B20489
:1019C0009093B304A093B404B093B504FF91EF9146
:1019D000BF91AF919F918F917F916F915F914F9147
:1019E0003F912F910F900FBE0F901F901895CF929F
:1019F000DF92EF92FF920F931F93CF93DF931F928B
:101A0000CDB7DEB77C01262F82E8860F8701065B03
:101A10001E4F823010F06B3149F4F8016081718102
:101A20008BE190E029830E94BD232981D701A05B2F
:101A3000BE4F3C9111964C911197822F90E0FC0182
:101A4000E327EE0FFF1FE851FF4F25913491C42E7D
:101A5000D12C2C253D252D933C93F801608171817B
:101A60000F90DF91CF911F910F91FF90EF90DF903A
:101A7000CF900C94BD2326E531E0DC01F9011D92E5
:101A80003197E9F7FC01E65BFE4F7183608338967E
:101A90005183408332972FEF3FEF3183208332977A
:101AA0003183208308952F923F924F925F926F92DD
:101AB0007F928F929F92AF92BF92CF92DF92EF92DE
:101AC000FF920F931F93CF93DF93CDB7DEB7C5552A
:101AD000D1090FB6F894DEBF0FBECDBF8C01865B77
:101AE0009E4F62969FAF8EAF629738019BEA691A4C
:101AF0009EEF790A5801ACEAAA1AAEEFBA0A780149
:101B0000B4EBEB1ABEEFFB0A6801E2EBCE1AEEEF84
:101B1000DE0A6296AEADBFAD62978D919C910E9438
:101B20007F238F3FBFEF9B0709F40FC1D3012C9197
:101B30002111DEC08E37910509F0CEC0F70120815A
:101B400031812231310508F4BBC0D6018D919C91C1
:101B5000883B904F09F0B4C0F801DE011896C80127
:101B6000069641914695403209F440E04D93E817BE
:101B7000F907B9F7F801868186958F708E87D801AD
:101B80001796FE013196CE0107964D91469540324B
:101B900009F440E04193E817F907B9F7F8013D96D9
:101BA000D8011D968C9186958F708F8329968FAC66
:101BB0002997912C61E070E0A7E02A2E808180FFB8
:101BC00010C028969FAE289729968FAE29978181BD
:101BD00090E02B969FAF8EAF2B97039709F070C0C4
:101BE0004EC0B8E09B1669F347E0949E2001112493
:101BF00066965FAE4EAE669781E090E0492D50E06C
:101C0000DF01A80FB91F3C90A32DA695A03211F0BB
:101C10003A2E01C0312C66964EAC5FAC6697480EEA
:101C2000591EA1E0B0E0AC0FBD1FA40DB51D1D965F
:101C30003C9201968730910519F737963080249EA3
:101C4000C001259E900D112444244394512C4C0E28
:101C50005D1E840D951DB32DB695BF705B2EDC0106
:101C600054965C92CB0101C0880F4A95EAF737FE83
:101C700002C0882A02C08095882293949FCF8281D7
:101C80002C968FAF2C97803FD9F433962250310990
:101C9000C8018E1B9F0B280F391F60963FAF2EAFD8
:101CA00060972E96FFAFEEAF2E97F801EE5AFE4FDB
:101CB0000190F081E02D309719F0CE010196099541
:101CC00081E0D5018C938FEF9FEFF60191838083A4
:101CD000D7011D921C921DCF8F37910511F4F5018C
:101CE00032C08B31910521F481E0D3018C9311CF67
:101CF000F5012081222331F1D7012D913C912A3425
:101D0000B1E03B07F0F4A9014F5F5F4FF70151834A
:101D10004083F801E20FF31F8083D6012D913C919F
:101D2000F901E827FF27EE0FFF1FE851FF4F8591CC
:101D30009491232F332728273927F60131832083D5
:101D400001C01082F3011082E4CECB5ADF4F0FB6F0
:101D5000F894DEBF0FBECDBFDF91CF911F910F91E1
:101D6000FF90EF90DF90CF90BF90AF909F908F90BB
:101D70007F906F905F904F903F902F9008958F923B
:101D80009F92AF92BF92CF92DF92EF92FF920F930A
:101D90001F93CF93DF938C014B015A016C0180EBB1
:101DA000C81A8EEFD80A8FEF9FEFF60191838083D8
:101DB0007801F6EBEF1AFEEFFF0AF70160817181FF
:101DC0008EE790E00E94BD23E401A80CB91CCA155F
:101DD000DB0529F06991C8010E94F70CF8CFF601E4
:101DE0006081C1816095C8010E94F70C6C2F6095DD
:101DF000C8010E94F70CF701608171818EE790E0C5
:101E0000DF91CF911F910F91FF90EF90DF90CF90D6
:101E1000BF90AF909F908F900C94BD232F923F92D4
:101E20004F925F926F927F928F929F92AF92BF92EA
:101E3000CF92DF92EF92FF920F931F93CF93DF9396
:101E4000CDB7DEB729970FB6F894DEBF0FBECDBF72
:101E5000998788876B014A012C833D835C0180EB65
:101E6000A81A8EEFB80A8FEF9FEFF5019183808358
:101E700028843984F6EB2F1AFEEF3F0AF1016081C6
:101E800071818EE790E00E94BD237601C12CD12C98
:101E9000C40101979B838A83C814D90409F457C0ED
:101EA00091E09983EA81FB81CE16DF0609F0198261
:101EB000F70101900020E9F731973F016E187F0884
:101EC000F7E06F16710418F086E0682E712C970108
:101ED000260D371D27014216530689F0F201819124
:101EE0002F0190E02E833F830E946623682F660FA8
:101EF000888599850E94F70C3F812E81ECCFF6E012
:101F00006F16710489F489818066F7016681660F16
:101F1000682B888599850E94F70CFFEFCF1ADF0A9E
:101F200087E0E80EF11CB8CF412C512CE6E0F0E040
:101F3000E619F7093F014614570428F760E488853D
:101F400099850E94F70C9FEF491A590AF4CF63E074
:101F5000888599850E94F70C60EF888599850E9495
:101F6000F70CEC80FD800E0D1F1DE016F10641F010
:101F7000F70161917F01888599850E94F70CF5CF63
:101F8000F501608111816095888599850E94F70C23
:101F9000612F6095888599850E94F70CF101608119
:101FA00071818EE790E029960FB6F894DEBF0FBEE0
:101FB000CDBFDF91CF911F910F91FF90EF90DF90F8
:101FC000CF90BF90AF909F908F907F906F905F90D9
:101FD0004F903F902F900C94BD2390931E068093BA
:101FE0001D065093B7044093B60470932006609387
:101FF0001F060895EF92FF920F931F93CF93DF93E5
:10200000EC016091B6047091B70480EC90E00E94FE
:10201000BD236091B6047091B70480E090E00E9407
:10202000BD238E017E0184EBE81A8EEFF80AF701DA
:1020300020813181225031096091B6047091B7043A
:10204000C8018C1B9D0B8217930708F5F80181913D
:102050008F01803C59F48BED90E00E94BD2360918C
:10206000B6047091B7048CED90E00EC08B3D59F42E
:102070008BED90E00E94BD236091B6047091B7048F
:102080008DED90E001C090E00E94BD23D0CF80ECA8
:1020900090E0DF91CF911F910F91FF90EF900C9402
:1020A000BD234F925F926F927F928F929F92AF92D9
:1020B000BF92EF92FF920F931F93CF93DF93EC01A8
:1020C0008B017A01E0911F06F09120068189811130
:1020D00045C00E94382390910001891798F4A70108
:1020E000B801CE01DF91CF911F910F91FF90EF903A
:1020F000BF90AF909F908F907F906F905F904F9028
:102100000C94BF0E8FB7F8948090B2049090B304F3
:10211000A090B404B090B5048FBF2091010130911C
:1021200002014091030150910401AAE0B0E00E9435
:102130004B212FB7F8944090B2045090B3046090B4
:10214000B4047090B5042FBF481859086A087B087A
:10215000461657066806790664F3B4CFE0911F0669
:10216000F09120068189882309F4ACCF80911D0667
:1021700090911E060E94530DE0911F06F0912006DB
:10218000E853FF4F80819181892B41F311821082A6
:10219000DF91CF911F910F91FF90EF90BF90AF9083
:1021A0009F908F907F906F905F904F900895909147
:1021B00021069923A1F0803C01F580910D01811148
:1021C00011C010922106409122065091230664E925
:1021D00072E080911D0690911E060C945110803C77
:1021E00009F07BC081E0809321068EEF80930D0182
:1021F0001092230610922206089520912206309113
:1022000023062A3491E0390708F067C090910D0148
:102210002115310531F49E3F21F48F7080930D011B
:10222000089591111FC08B3D21F481E080931C061D
:10223000089590911C06992349F08C3D21F08D3D25
:1022400019F48BED01C080EC10921C06A9014F5FC0
:102250005F4F5093230640932206F901EC56FD4F41
:1022600080830895913079F4282F30E0AAE0B0E01F
:102270000E9435216093090170930A0180930B013C
:1022800090930C010895943089F42AE0829FC00154
:102290001124AA2797FDA095BA2F8093050190934A
:1022A0000601A0930701B09308010895933089F4C3
:1022B0002AE0829FC0011124AA2797FDA095BA2F7A
:1022C0008093010190930201A0930301B093040154
:1022D0000895923011F48093000108956FEF8EE21B
:1022E00090E00E941B2680913201882341F083E117
:1022F0009EE09F938F930E94F5230F900F90809103
:10230000320181110CC08091E703811108C080E186
:102310009EE09F938F930E94F5230F900F90089556
:10232000CF938EE290E00E94FD25893609F0E3C04C
:1023300046E050E068E270E08CE291E00E94ED251A
:1023400046E050E062E270E086E291E00E94ED2516
:1023500046E050E06CE170E080E291E00E94ED2503
:1023600046E050E066E170E088E191E00E94ED25F2
:1023700085E190E00E94FD2590E09093E403809336
:10238000E30384E190E00E94FD2590E09093E20356
:102390008093E10383E190E00E94FD2590E090931B
:1023A0001F0180931E0182E190E00E94FD2590E0D4
:1023B000909317018093160181E190E00E94FD2522
:1023C00091E0811101C090E09093370180E190E0AD
:1023D0000E94FD2591E0811101C090E090933601AB
:1023E0008FE090E00E94FD2591E0811101C090E016
:1023F000909335018EE090E00E94FD2591E08111DF
:1024000001C090E0909334018DE090E00E94FD25A2
:1024100091E0811101C090E0909333018CE090E055
:102420000E94FD25C1E0811101C0C0E0C0933201CE
:102430008BE090E00E94FD2591E0811101C090E0C9
:102440009093E7038AE090E00E94FD2580931301BA
:1024500089E090E00E94FD258093120188E090E0E1
:102460000E94FD258093110187E090E00E94FD25E8
:102470008093100186E090E00E94FD258093150175
:1024800085E090E00E94FD258093140184E090E0B7
:102490000E94FD2591E0811101C090E09093DE0340
:1024A00082E090E00E940526A0E0B0E08093090160
:1024B00090930A01A0930B01B0930C0180E090E08F
:1024C0000E940526A0E0B0E08093050190930601EC
:1024D000A0930701B0930801CC23C1F18091E603DA
:1024E0008823A1F18AEF9DE09F938F930E94F523AB
:1024F0000F900F902BC08091E603882381F080918C
:10250000E70381110CC080913201882341F081EDF5
:102510009DE09F938F930E94F5230F900F908091E1
:10252000E603882381F08091E70381110CC080913C
:102530003201811108C08EEC9DE09F938F930E9421
:10254000F5230F900F9081E08093E503CF910895DC
:1025500090931E0680931D060E94901181E0809347
:10256000E603809132018823A1F18AEA9EE09F93DD
:102570008F930E94F52389E99EE09F938F930E9499
:10258000F52382E89EE09F938F930E94F5230F909E
:102590000F900F900F900F900F908091E50388237C
:1025A00041F083E69EE09F938F930E94F5230F9066
:1025B0000F9086E59EE09F938F930E94F52385E41C
:1025C0009EE09F938F930E94F5230F900F900F90A2
:1025D0000F90089546E050E068E270E08CE291E0F0
:1025E0000E940B2646E050E062E270E086E291E055
:1025F0000E940B2646E050E06CE170E080E291E042
:102600000E940B2646E050E066E170E088E191E030
:102610000E940B266091E30385E190E00E941B2657
:102620006091E10384E190E00E941B2660911E010D
:1026300083E190E00E941B266091160182E190E008
:102640000E941B266091370181E190E00E941B26C9
:102650006091360180E190E00E941B266091350177
:102660008FE090E00E941B26609134018EE090E0A4
:102670000E941B26609133018DE090E00E941B2692
:10268000609132018CE090E00E941B266091E7038C
:102690008BE090E00E941B26609113018AE090E09D
:1026A0000E941B266091120189E090E00E941B2687
:1026B0006091110188E090E00E941B26609110015A
:1026C00087E090E00E941B266091150186E090E073
:1026D0000E941B266091140185E090E00E941B2659
:1026E0006091DE0384E090E00E941B266091090166
:1026F00070910A0182E090E00E942C266091050111
:102700007091060180E090E00E942C2669E68EE23E
:1027100090E00E941B2680913201882341F089EBD2
:102720009DE09F938F930E94F5230F900F908091CF
:10273000320181110CC08091E703811108C086EB42
:102740009DE09F938F930E94F5230F900F90089523
:102750000F931F93CF93DF939C01EA0186E0E6E29B
:10276000F1E0A2E4B6E001900D928A95E1F7809144
:10277000E1038093480696E0ECE2F1E0A1EAB6E0DE
:1027800001900D929A95E1F78091E3038093A7065B
:1027900096E0E0E2F1E0A9E4B6E001900D929A95AE
:1027A000E1F780911E0180934F0696E0E8E1F1E0A9
:1027B000A1EBB6E001900D929A95E1F78091160198
:1027C0008093B70697E0E2E4F6E0A4E2B6E0019079
:1027D0000D929A95E1F797E0E1EAF6E0ABE2B6E018
:1027E00001900D929A95E1F797E0E9E4F6E0A2E313
:1027F000B6E001900D929A95E1F797E0E1EBF6E0F3
:10280000A9E3B6E001900D929A95E1F78B0144E0BF
:1028100050E064E276E0CE010E940E0FDF91CF918E
:102820001F910F9108958F929F92AF92BF92CF9276
:10283000DF92EF92FF920F931F93CF93DF9300D01D
:1028400000D000D0CDB7DEB78C018091370188234E
:10285000F9F080913301882341F080EB9DE09F9354
:102860008F930E94F5230F900F90D80116968C91AC
:102870001F928F931F930F9385EA9DE09F938F93F1
:102880000E94F5230F900F900F900F900F900F90D4
:1028900080913601882301F180913301882341F032
:1028A0008FE99DE09F938F930E94F5230F900F90E7
:1028B000F80185851F928F93C80107969F938F9388
:1028C00084E99DE09F938F930E94F5230F900F90D2
:1028D0000F900F900F900F9080913501811105C0DE
:1028E00080913401811147C039C080913301882320
:1028F00041F08DE89DE09F938F930E94F5230F9008
:102900000F907801F4E1EF0EF11CC12CD12C58018D
:1029100026E4A20EB11C82E8882E8DE0982ED50107
:102920008C9190E0C816D906DCF6D7018C911F92E5
:102930008F93C70106979F938F939F928F920E94C8
:10294000F523BFEFCB1ADB0AE7E0EE0EF11C0F9088
:102950000F900F900F900F900F90E1CF88E79DE0C0
:102960009F938F930E94F5230F900F908091DE0329
:10297000811134C02FC180913301F801E35BFF4F17
:102980006F01882371F081818F9380818F938BE712
:102990009DE09F938F930E94F5230F900F900F90CF
:1029A0000F90E12CF12C5801FBE4AF0EB11CF601A5
:1029B00080819181E816F90688F66091BE067091D3
:1029C000BF06D501ED91FC91EE0DFF1D808190E0D9
:1029D0000E94BD23BFEFEB1AFB0AE9CFF801E35BCE
:1029E000FF4FA081B181AC30B10508F4F3C032973C
:1029F0000190F081E02D5D01AE0EBF1E40E050E081
:102A0000C12CD12CBE016F5F7F4FD5018E915D012E
:102A10008B3731F04F5F5F4F47305105B1F710C032
:102A2000CB019D01D901FD909D01DC01FD92CD01FD
:102A30007D01E61AF70A4E155F05A0F76A01EACF95
:102A4000C114D10409F4C6C081E090E041E0DF0187
:102A5000A80FB91F3C91DC01A55DBE4F2C91321728
:102A600019F087E090E040E00196873091057CF313
:102A700020E030E0DF01A80FB91F5C915D3209F45E
:102A80009C0101968A309105A9F72115310599F02D
:102A9000E20FF31F82812091E3033091E40380323F
:102AA00021F4818190E0C09702C090E08697821760
:102AB000930709F08FC0442309F48CC05601BEE08F
:102AC000AB0EB11CC5010E94BF217C01FC013196F7
:102AD0000A9620E22193E817F907E1F7B801E0E050
:102AE000F0E080E090E0DB012D91BD01222339F080
:102AF000A701480F591FDA0111962C9331960196C0
:102B00008630910581F7D80116969C91992369F03A
:102B1000EE0DFF1D8DE281839A3018F4905D928353
:102B200004C081E382839A5D93838AE3F701808303
:102B3000828781E6838783E684878BE685873E9656
:102B400080E090E00196A1E0B0E0AC0FBD1FA80FBF
:102B5000B91F2C9121938C159D05A4F38FB7F89480
:102B60004091B2045091B3046091B4047091B504E3
:102B70008FBF2FB7F8948091B2049091B304A091C5
:102B8000B404B091B5042FBF841B950BA60BB70BF3
:102B90008C359444A105B10560F340911D06509118
:102BA0001E06B501C7010E94A813C70126960FB6DD
:102BB000F894DEBF0FBECDBFDF91CF911F910F9173
:102BC000FF90EF90DF90CF90BF90AF909F908F904D
:102BD0000C94542226960FB6F894DEBF0FBECDBFDC
:102BE000DF91CF911F910F91FF90EF90DF90CF90E9
:102BF000BF90AF909F908F9008958F929F92AF92C9
:102C0000BF92CF92DF92EF92FF920F931F93CF93D9
:102C1000DF934C017B015A016B0184E1C80ED11C8A
:102C2000009113010A3090F4809112018A3070F4FF
:102C3000809111018A3050F480911001893030F474
:102C40006B018BE1C80ED11C11E001C010E0C60180
:102C50000E94BF21EC018DE3888380911501898753
:102C6000809114018B8B88E0E9E9F6E0DE01119692
:102C700001900D928A95E1F789E0E8EAF6E0DE013D
:102C80001A9601900D928A95E1F7111103C0CE01B9
:102C9000449616C080E58C8B88E48D8B87E48E8B00
:102CA000005D0F8B80911201805D888F80911101F2
:102CB000805D898F80911001805D8A8FCE014B9657
:102CC000E114F10421F0A701B4010E946E23A501D3
:102CD000B601CE010E94A813CE01DF91CF911F91C2
:102CE0000F91FF90EF90DF90CF90BF90AF909F90AB
:102CF0008F900C9454228F929F92AF92BF92CF925A
:102D0000DF92EF92FF920F931F93CF93DF937C019B
:102D10006A01EB016434710510F0C3E4D0E08E0168
:102D2000015F1F4FC8010E94BF215C018AE3F501CA
:102D3000808387E090E020E030E0019769F0F901BE
:102D4000E05BF94F40814423C1F32F5F3F4FF50112
:102D5000E20FF31F4083F1CF80910E0190910F019C
:102D60008F3FFFEF9F0779F0F501E20FF31F4DE270
:102D700041838A3091054CF42E5F3F4FF501E20FFD
:102D8000F31F805D808380E209C091E392832D5F11
:102D90003F4FF501E20FF31F8A5DF4CF2930310573
:102DA0003CF42F5F3F4FF501E20FF31F8083F6CF16
:102DB000F501E20FF31F8AE38183209781F0AE01D2
:102DC000B701C5010B960E946E23AE01B70186E5DF
:102DD00096E00E946E23D0934106C09340068091F6
:102DE000DF039091E0030196883E23E092072CF4E4
:102DF0009093E0038093DF0304C01092E0031092ED
:102E0000DF03CA0DDB1D8BE78B872091DF03309139
:102E1000E0038AE0882E912CC901B4010E9456215A
:102E2000FC0194E6E92EF12CC901B7010E9456215C
:102E30008E1B9F0BB4010E945621AB01C901861B5A
:102E4000970B8E1B9F0BB7010E945621605D6C870C
:102E5000405D4D87E05DEE87A601B801C5010E9487
:102E6000A813C501DF91CF911F910F91FF90EF90B3
:102E7000DF90CF90BF90AF909F908F900C94542292
:102E80002091DF033091E003215031093093E003BA
:102E90002093DF036091400670914106AC0186E506
:102EA00096E00C947B1683E199E09F938F930E94A8
:102EB000F5238091E4038F938091E3038F938CE259
:102EC00091E09F938F9380E099E09F938F930E946E
:102ED000F5238091E2038F938091E1038F9386E243
:102EE00091E09F938F938AEE98E09F938F930E9437
:102EF000F52380911F018F9380911E018F9380E2B3
:102F000091E09F938F938AED98E09F938F930E9417
:102F1000F523809117018F93809116018F9388E19B
:102F200091E09F938F938AEC98E09F938F930E94F8
:102F3000F5238DB79EB74A960FB6F8949EBF0FBE85
:102F40008DBF8091DE03882319F083EB98E002C0E7
:102F50008BE998E09F938F930E94F5230F900F9039
:102F6000809113018A3061F01F928F9380E998E07D
:102F70009F938F930E94F5230F900F900F900F90C7
:102F8000809112018A3061F01F928F9384E898E05B
:102F90009F938F930E94F5230F900F900F900F90A7
:102FA000809111018A3061F01F928F938AE798E037
:102FB0009F938F930E94F5230F900F900F900F9087
:102FC000809110018A3061F01F928F9389E698E01A
:102FD0009F938F930E94F5230F900F900F900F9067
:102FE000809115018C3541F480E598E09F938F9393
:102FF0000E94F5230F900F90809115018F3241F4BC
:1030000088E398E09F938F930E94F5230F900F9091
:10301000809114011F928F938CE298E09F938F937D
:103020000E94F52380910C018F9380910B018F9367
:1030300080910A018F93809109018F938AE198E032
:103040009F938F930E94F523809108018F93809125
:1030500007018F93809106018F93809105018F93D3
:103060008CE098E09F938F930E94F5238DB79EB7D5
:1030700040960FB6F8949EBF0FBE8DBF089588EEA0
:1030800097E09F938F930E94F52386ED97E09F939F
:103090008F930E94F5238BEB97E09F938F930E9471
:1030A000F52382E897E09F938F930E94F52384E6AF
:1030B00097E09F938F930E94F52387E497E09F9377
:1030C0008F930E94F52383E297E09F938F930E9452
:1030D000F52385E097E09F938F930E94F52386EE7A
:1030E00096E09F938F930E94F5238DEC96E09F933B
:1030F0008F930E94F5238DEA96E09F938F930E9411
:10310000F52383E996E09F938F930E94F52388E748
:1031100096E09F938F930E94F52385E496E09F931A
:103120008F930E94F52381E196E09F938F930E94F5
:10313000F52384EF95E09F938F930E94F5238DB73D
:103140009EB780960FB6F8949EBF0FBE8DBF81EDDF
:1031500095E09F938F930E94F52380EB95E09F93DA
:103160008F930E94F52388E895E09F938F930E94A8
:10317000F5238FE695E09F938F930E94F5238AE3D2
:1031800095E09F938F930E94F52380E195E09F93B4
:103190008F930E94F5238AEE94E09F938F930E9471
:1031A000F5238CEC94E09F938F930E94F52383EAA0
:1031B00094E09F938F930E94F52387E894E09F9378
:1031C0008F930E94F5238BE694E09F938F930E9448
:1031D000F5238EE494E09F938F930E94F52381E37F
:1031E00094E09F938F930E94F52383E194E09F9353
:1031F0008F930E94F52384EF93E09F938F930E9417
:10320000F52385ED93E09F938F930E94F5238DB76F
:103210009EB780960FB6F8949EBF0FBE8DBF82EB0F
:1032200093E09F938F930E94F52386E893E09F930A
:103230008F930E94F52388E693E09F938F930E94DB
:10324000F5238AE493E09F938F930E94F5238BE20A
:1032500093E09F938F930E94F5238CE093E09F93DC
:103260008F930E94F52388EE92E09F938F930E94A4
:10327000F5238DB79EB70E960FB6F8949EBF0FBE7E
:103280008DBF0895EF92FF920F931F93CF93DF931B
:1032900000D000D0CDB7DEB76115710509F47CC749
:1032A0009B018C01DC019C91913209F56230710522
:1032B00008F450C661507109C80101960E94A81314
:1032C00080913201882341F08BE69DE09F938F939C
:1032D0000E94F5230F900F908091320181115CC7FD
:1032E0008091E703811158C788E69DE049C6903474
:1032F000E9F461507109C80101960E94FD158091A1
:103300003201882341F082E59DE09F938F930E94D4
:10331000F5230F900F908091320181113DC780916C
:10332000E703811139C78FE49DE02AC69332E9F49F
:1033300061507109C80101960E947B16809132018B
:10334000882341F081E49DE09F938F930E94F523B1
:103350000F900F908091320181111EC78091E70379
:1033600081111AC78EE39DE00BC6983619F40E94AE
:103370003F1812C7983419F40E9453170DC793359C
:1033800019F40E94EA1208C7933419F40E946E11CE
:1033900003C79C3419F40E949011FEC6933609F0BD
:1033A00050C06430710508F4D5C54CE251E00F5FA0
:1033B0001F4F61507109E0E0F0E0E630F105A1F047
:1033C000D8019D918D01992339F09A3029F09D30D3
:1033D00019F0DA019C9302C0DA011C9231964F5F1A
:1033E0005F4FE617F70749F7E45DFE4FB1E0E233C0
:1033F000FB0711F01192FACF809132018823B1F0CE
:103400008091E4038F938091E3038F938CE291E0AA
:103410009F938F938BE29DE09F938F930E94F52360
:103420000F900F900F900F900F900F90809132019E
:103430008111B2C68091E7038111AEC688E29DE09A
:103440009FC5943609F051C06430710508F482C5F7
:10345000E6E2F1E0D80111962150310940E050E058
:1034600046305105A1F09D91992331F09A3021F019
:103470009D3011F0908301C010824F5F5F4F3196F5
:103480004217530769F7F901EA5DFE4F03C026E0D2
:1034900030E0F9CF21E0EC32F20711F01192FACFCF
:1034A000809132018823B1F08091E2038F93809163
:1034B000E1038F9386E291E09F938F9382E19DE0F9
:1034C0009F938F930E94F5230F900F900F900F9072
:1034D0000F900F908091320181115EC68091E703B9
:1034E00081115AC68FE09DE04BC5913309F050C061
:1034F0006230710508F42EC540E251E00F5F1F4FA6
:1035000061507109E0E0F0E0E630F105A1F0D8018A
:103510009D918D01992339F09A3029F09D3019F051
:10352000DA019C9302C0DA011C9231964F5F5F4F23
:10353000E617F70749F7E05EFE4FB1E0E632FB071A
:1035400011F01192FACF809132018823B1F080916D
:103550001F018F9380911E018F9380E291E09F93D2
:103560008F938FEF9CE09F938F930E94F5230F9092
:103570000F900F900F900F900F908091320181115A
:103580000BC68091E703811107C68CEF9CE0F8C45D
:10359000923309F051C06230710508F4DBC4E8E1F0
:1035A000F1E0D80111962150310940E050E0463059
:1035B0005105A1F09D91992331F09A3021F09D3071
:1035C00011F0908301C010824F5F5F4F3196421718
:1035D000530769F7F901E85EFE4F03C026E030E0CB
:1035E000F9CF21E0EE31F20711F01192FACF80917C
:1035F00032018823B1F0809117018F9380911601D9
:103600008F9388E191E09F938F938CEE9CE09F9342
:103610008F930E94F5230F900F900F900F900F90B3
:103620000F90809132018111B7C58091E70381111C
:10363000B3C589EE9CE0A4C4933709F038C1633068
:10364000710508F487C47B0181E0E81AF108D8010C
:1036500011968C911197833609F046C012968C9181
:10366000B2E0EB16F10461F0F80193812FEC290F21
:10367000293030F4813320F0892F90E0869706C0FE
:103680009FEC980F993030F490E0C0979093E4034A
:103690008093E303809132018823B1F08091E403A9
:1036A0008F938091E3038F938CE291E09F938F93AC
:1036B00086ED9CE09F938F930E94F5230F900F90CF
:1036C0000F900F900F900F908091320181110CC0DC
:1036D0008091E703811108C083ED9CE09F938F9355
:1036E0000E94F5230F900F90D80111968C9111979D
:1036F000843609F046C012968C91B2E0EB16F104C4
:1037000061F0F80193812FEC290F293030F48133D7
:1037100020F0892F90E0869706C09FEC980F993093
:1037200030F490E0C0979093E2038093E10380919E
:1037300032018823B1F08091E2038F938091E103FD
:103740008F9386E291E09F938F938DEB9CE09F9304
:103750008F930E94F5230F900F900F900F900F9072
:103760000F908091320181110CC08091E70381118B
:1037700008C08AEB9CE09F938F930E94F5230F90E3
:103780000F90D80111968C911197813309F046C0A2
:1037900012968C91B2E0EB16F10461F0F80193817E
:1037A0002FEC290F293030F4813320F0892F90E05D
:1037B000869706C09FEC980F993030F490E0C09740
:1037C00090931F0180931E01809132018823B1F0F4
:1037D00080911F018F9380911E018F9380E291E071
:1037E0009F938F938AEA9CE09F938F930E94F52387
:1037F0000F900F900F900F900F900F9080913201CB
:1038000081110CC08091E703811108C087EA9CE018
:103810009F938F930E94F5230F900F90D8011196DC
:103820008C911197823309F0B7C413968C91B2E052
:10383000EB16F10459F09FEC980F993038F4F80129
:103840009281913318F090E0869708C081538930B7
:1038500048F4D80112968C9190E0C097909317018C
:1038600080931601809132018823B1F08091170175
:103870008F93809116018F9388E191E09F938F93AE
:1038800087E99CE09F938F930E94F5230F900F9000
:103890000F900F900F900F908091320181117CC496
:1038A0008091E703811178C484E99CE069C3903773
:1038B00009F037C16330710508F44CC3F801818108
:1038C0008337C9F59281809132019133C1F491E03F
:1038D00090933701882341F081E89CE09F938F9378
:1038E0000E94F5230F900F9080913201811123C027
:1038F0008091E70381111FC08EE79CE016C01092F3
:103900003701882341F08AE69CE09F938F930E94C1
:10391000F5230F900F908091320181110CC080919E
:10392000E703811108C087E69CE09F938F930E9474
:10393000F5230F900F90D80111968C911197843632
:10394000D1F512969C91809132019133C1F491E0AE
:1039500090933601882341F084E59CE09F938F93F8
:103960000E94F5230F900F9080913201811123C0A6
:103970008091E70381111FC081E59CE016C0109281
:103980003601882341F08DE39CE09F938F930E9442
:10399000F5230F900F908091320181110CC080911E
:1039A000E703811108C08AE39CE09F938F930E94F4
:1039B000F5230F900F90F80181818037C9F592812E
:1039C000809132019133C1F491E0909335018823C5
:1039D00041F086E29CE09F938F930E94F5230F9025
:1039E0000F9080913201811123C08091E7038111F2
:1039F0001FC083E29CE016C010923501882341F07D
:103A00008EE09CE09F938F930E94F5230F900F9080
:103A10008091320181110CC08091E703811108C0AF
:103A20008BE09CE09F938F930E94F5230F900F9063
:103A3000D80111968C9111978D36D1F512969C91E3
:103A4000809132019133C1F491E090933401882345
:103A500041F087EF9BE09F938F930E94F5230F9097
:103A60000F9080913201811123C08091E703811171
:103A70001FC084EF9BE016C010923401882341F0F0
:103A80008FED9BE09F938F930E94F5230F900F90F3
:103A90008091320181110CC08091E703811108C02F
:103AA0008CED9BE09F938F930E94F5230F900F90D6
:103AB000F8018181893609F06FC3928180913201CA
:103AC0009133C1F491E090933301882341F088EC65
:103AD0009BE09F938F930E94F5230F900F9080910E
:103AE0003201811159C38091E703811155C385ECDF
:103AF0009BE046C210923301882341F080EB9BE0AB
:103B00009F938F930E94F5230F900F908091320125
:103B1000811142C38091E70381113EC38DEA9BE08E
:103B20002FC2963781F4D80111968C91813331F4EC
:103B300081E08093320187E99BE022C2109232013A
:103B400080E89BE01DC2963589F4F80181818133BC
:103B500041F481E08093E703109232018BE69BE011
:103B60000FC21092E70385E59BE00AC29C3609F07C
:103B700068C06330710508F4EDC1D80111968C91CD
:103B800011978C3609F003C26150710912968C911D
:103B9000813651F56A30710508F4FEC288E0F801FB
:103BA0003396A9E9B6E001900D928A95E1F78091EC
:103BB0003201882371F089E996E09F938F938FE318
:103BC0009BE09F938F930E94F5230F900F900F908F
:103BD0000F90809132018111DFC28091E703811142
:103BE000DBC28CE39BE0CCC18F3609F0D5C26B30D1
:103BF000710508F4D1C289E0F8013396A8EAB6E06D
:103C000001900D928A95E1F780913201882371F03D
:103C100088EA96E09F938F9384E29BE09F938F9333
:103C20000E94F5230F900F900F900F90809132011A
:103C30008111B2C28091E7038111AEC281E29BE0A3
:103C40009FC19D3609F021C16230710508F482C11F
:103C500061507109F8018181833609F067C06130D4
:103C6000710509F499C240E556E00E5F1F4F61509F
:103C70007109E0E0F0E0E617F70719F4E05BF94FAF
:103C800015C0E630F105D1F3D8019D918D0199233E
:103C900039F09A3029F09D3019F0DA019C9302C076
:103CA000DA011C9231964F5F5F4FE5CFB6E0E63503
:103CB000FB0711F01192FACF80913201882359F15C
:103CC00080E596E09F938F9380E39AE09F938F9394
:103CD0000E94F52380910E0190910F010F900F909B
:103CE0000F900F908F3FEFEF9E0769F09F938F9398
:103CF0008BE29AE09F938F930E94F5230F900F9091
:103D00000F900F9008C089E29AE09F938F930E94D2
:103D1000F5230F900F908091320181113DC2809167
:103D2000E703811139C286E29AE02AC1833709F09C
:103D300059C06130710509F42FC26430710520F05B
:103D4000838190E0869704C0F801828190E0C0975B
:103D500090930F0180930E0180910E0190910F01BD
:103D6000409730F08FEF9FEF90930F0180930E01FB
:103D700080913201882359F180E596E09F938F93DB
:103D80008EE09AE09F938F930E94F52380910E011D
:103D900090910F010F900F900F900F908F3FFFEFBA
:103DA0009F0769F09F938F9389E09AE09F938F9389
:103DB0000E94F5230F900F900F900F9008C087E09E
:103DC0009AE09F938F930E94F5230F900F9080911C
:103DD00032018111E1C18091E7038111DDC184E0ED
:103DE0009AE0CEC08237D1F4CA010E944017809178
:103DF0003201882341F08EEE99E09F938F930E94C9
:103E0000F5230F900F90809132018111C5C18091EF
:103E1000E7038111C1C18BEE99E0B2C0813609F090
:103E2000BBC19281809132019133C1F491E09093B2
:103E3000DE03882341F081ED99E09F938F930E94E8
:103E4000F5230F900F90809132018111A5C18091CF
:103E5000E7038111A1C18EEC99E092C01092DE03BC
:103E6000882341F083EB99E09F938F930E94F52381
:103E70000F900F908091320181118EC18091E703E4
:103E800081118AC180EB99E07BC0973761F5623080
:103E9000710508F45FC0AB0141505109B8016F5F73
:103EA0007F4FCE0101960E946E23CE0101960E94A3
:103EB00048238031B7E29B0798F4AA2797FDA09585
:103EC000BA2F8093090190930A01A0930B01B0933C
:103ED0000C01BF93AF939F938F9389E999E02CC016
:103EE00086E799E04DC09735A9F56230710590F1EC
:103EF000AB0141505109B8016F5F7F4FCE01019670
:103F00000E946E23CE0101960E9448238031E7E291
:103F10009E07E8F4AA2797FDA095BA2F8093050184
:103F200090930601A0930701B0930801BF93AF934C
:103F30009F938F9380E699E09F938F930E94F52340
:103F40000F900F900F900F900F900F9025C18EE360
:103F500099E016C080913201882341F086E299E011
:103F60009F938F930E94F5230F900F9080913201C1
:103F7000811112C18091E70381110EC183E299E0A2
:103F80009F938F930E94F5230F900F9005C1803768
:103F900031F5F801828180538A3008F0FDC08093AA
:103FA000130190913201992379F0889FC001112467
:103FB0009F938F938FE09BE09F938F930E94F523B5
:103FC0000F900F900F900F90809132018111E4C0FB
:103FD0008091E7038111E0C08CE09BE0D1CF88366F
:103FE000C9F5D80112968C9180538A3008F0D4C05C
:103FF0008093120190913201992309F1A1E0B0E080
:1040000002C0AA0FBB1F8A95E2F728EE33E00E9498
:10401000442128E431E040E050E00E948C215F938D
:104020004F933F932F938CEE9AE09F938F930E9430
:10403000F5230F900F900F900F900F900F9080919D
:1040400032018111A9C08091E7038111A5C089EED9
:104050009AE096CF873619F5F801828180538A302D
:1040600008F09AC08093110190913201992361F078
:104070001F928F9387ED9AE09F938F930E94F52371
:104080000F900F900F900F9080913201811184C09A
:104090008091E703811180C084ED9AE071CF84366E
:1040A000D9F5D80112968C9180538A3008F074C0EB
:1040B000893009F488E080931001809132018111E8
:1040C0000CC08091E703811108C081ED9AE09F93B5
:1040D0008F930E94F5230F900F90809132018823D7
:1040E00009F45AC080911001811108C088EB9AE050
:1040F0009F938F930E94F5230F900F908091100152
:10410000882309F449C0BDE28B9FC00111249F930D
:104110008F938EE99AE00EC08337A9F4F80182816B
:1041200080931401909132019923B1F11F928F93E2
:104130008CE89AE09F938F930E94F5230F900F9045
:104140000F900F9029C0843739F5D80112969C91B1
:1041500080913201913641F49CE5909315018823BA
:1041600081F08BE69AE007C09FE2909315018823C7
:1041700041F08BE49AE09F938F930E94F5230F9078
:104180000F9080913201811107C08091E703811166
:1041900003C088E49AE0F4CE0F900F900F900F9038
:1041A000DF91CF911F910F91FF90EF9008950E94A2
:1041B0008B070E947D076B017C01C1E084EC94E0D9
:1041C0000E94530D80914201811125C00E94F70782
:1041D000882309F10E940108282F30E0309346011E
:1041E000209345012091430130914401F901E95B9D
:1041F000FE4FA9014F5F5F4F80835093440140936E
:1042000043012934314010F0C09342010E947D07E0
:104210006B017C0114C08091430190914401892B72
:1042200071F00E947D07DC01CB018C199D09AE095C
:10423000BF094597A105B10514F0C09342018091D3
:104240004201882309F4BACF60914301709144017F
:1042500044EC54E087E491E00E944219109242013C
:104260001092440110924301A9CFA29FB001B39FC5
:10427000C001A39F700D811D1124911DB29F700D6F
:10428000811D1124911D08950E943521B7FF0895C5
:10429000821B930B08950E943521A59F900DB49F1A
:1042A000900DA49F800D911D1124089597FB072E5A
:1042B00016F4009407D077FD09D00E94AB2107FCCB
:1042C00005D03EF4909581959F4F08957095619526
:1042D0007F4F0895A1E21A2EAA1BBB1BFD010DC042
:1042E000AA1FBB1FEE1FFF1FA217B307E407F507A6
:1042F00020F0A21BB30BE40BF50B661F771F881F82
:10430000991F1A9469F760957095809590959B0117
:10431000AC01BD01CF010895052E97FB1EF400945A
:104320000E94A32157FD07D00E946A2107FC03D0F9
:104330004EF40C94A32150954095309521953F4F14
:104340004F4F5F4F089590958095709561957F4F81
:104350008F4F9F4F0895AA1BBB1B51E107C0AA1F97
:10436000BB1FA617B70710F0A61BB70B881F991F16
:104370005A95A9F780959095BC01CD010895CF93EA
:10438000DF938230910510F482E090E0E091BA066C
:10439000F091BB0620E030E0C0E0D0E0309711F1B2
:1043A0004081518148175907C0F04817590761F4F7
:1043B00082819381209719F09B838A832BC09093ED
:1043C000BB068093BA0626C02115310519F04217A5
:1043D000530718F49A01BE01DF01EF010280F38157
:1043E000E02DDCCF2115310509F1281B390B2430D4
:1043F000310590F412968D919C911397611571057A
:1044000021F0FB019383828304C09093BB068093C9
:10441000BA06FD01329644C0FD01E20FF31F8193FD
:104420009193225031092D933C933AC02091B806C4
:104430003091B906232B41F420913A0130913B0190
:104440003093B9062093B806209138013091390194
:104450002115310541F42DB73EB740913C015091F3
:104460003D01241B350BE091B806F091B906E21727
:10447000F307A0F42E1B3F0B2817390778F0AC0187
:104480004E5F5F4F2417350748F04E0F5F1F509364
:10449000B9064093B8068193919302C0E0E0F0E042
:1044A000CF01DF91CF9108950F931F93CF93DF93A7
:1044B000009709F48CC0FC0132971382128200919C
:1044C000BA061091BB060115110581F420813181D6
:1044D000820F931F2091B8063091B906281739072B
:1044E00079F5F093B906E093B80671C0D80140E0C1
:1044F00050E0AE17BF0750F412962D913C911397E0
:10450000AD012115310509F1D901F3CF9D01DA0182
:104510003383228360817181860F971F82179307EF
:1045200069F4EC0128813981260F371F2E5F3F4F38
:10453000318320838A819B8193838283452B29F455
:10454000F093BB06E093BA0642C01396FC93EE9339
:104550001297ED01499159919E01240F351FE217E1
:10456000F30771F480819181840F951F0296119653
:104570009C938E938281938113969C938E93129732
:10458000E0E0F0E0D80112968D919C91139700978E
:1045900019F0F8018C01F6CF8D919C9198012E5F56
:1045A0003F4F820F931F2091B8063091B90628170C
:1045B000390769F4309729F41092BB061092BA06B5
:1045C00002C0138212821093B9060093B806DF91DD
:1045D000CF911F910F9108958F929F92AF92BF92AA
:1045E000CF92DF92EF92FF92CF93DF93EC0168813D
:1045F00079818A819B81611571058105910521F47D
:1046000064E279ED8BE597E02DE133EF41E050E096
:104610000E948C2149015A019B01AC01A7EAB1E437
:104620000E944B216B017C01ACEEB4EFA50194011B
:104630000E94A926DC01CB018C0D9D1DAE1DBF1D66
:10464000B7FF03C00197A109B04888839983AA8363
:10465000BB839F77DF91CF91FF90EF90DF90CF905A
:10466000BF90AF909F908F9008950E94EC22089584
:104670008EE391E00E94EC220895A0E0B0E08093E8
:104680003E0190933F01A0934001B09341010895F2
:10469000FC0188279927E89421912032E9F32930F9
:1046A00010F02E30C8F32B3241F02D3239F46894DB
:1046B00004C00E947723820F911D219120532A303C
:1046C000C0F31EF4909581959F4F08959111089520
:1046D00081568A5108F4805285580895FB01DC0107
:1046E00002C001900D9241505040D8F708957AE0F1
:1046F000979F902D879F802D910D11240895CF9322
:10470000DF93EC012B8120FF33C026FF0AC02F7BF3
:104710002B838E819F8101969F838E838A8190E077
:1047200029C022FF0FC0E881F9818081992787FD88
:104730009095009719F420622B831AC03196F98363
:10474000E8830EC0EA85FB85099597FF09C02B8198
:10475000019611F080E201C080E1822B8B8308C0BA
:104760002E813F812F5F3F4F3F832E83992702C0C9
:104770008FEF9FEFDF91CF9108950F931F93CF930A
:10478000DF93FB01238121FD03C08FEF9FEF28C042
:1047900022FF16C046815781248135814217530775
:1047A00044F4A081B1819D012F5F3F4F318320836D
:1047B0008C93268137812F5F3F4F3783268310C02C
:1047C000EB01092F182F0084F185E02D0995892B25
:1047D000E1F68E819F8101969F838E83812F902F9A
:1047E000DF91CF911F910F910895A0E0B0E0EBEF22
:1047F000F3E20C94BC26AE01495F5F4FDA016D9184
:104800007D91AD010CEB16E0F80182819381DC0112
:1048100013962C911397286013962C930E941B24B7
:10482000D8011296ED91FC9113972381277F238362
:10483000E4E00C94D826ACE0B0E0E1E2F4E20C94C1
:10484000AE267C016B018A01FC01178216828381EE
:1048500081FFBDC1CE0101964C01F7019381F601A4
:1048600093FD859193FF81916F01882309F4ABC17A
:10487000853239F493FD859193FF81916F018532E3
:1048800029F4B70190E00E94BD23E7CF512C312CD1
:1048900020E02032A0F48B3269F030F4803259F0FD
:1048A000833269F420612CC08D3239F0803339F4C1
:1048B000216026C02260246023C0286021C027FD1B
:1048C00027C030ED380F3A3078F426FF06C0FAE002
:1048D0005F9E300D1124532E13C08AE0389E300D98
:1048E0001124332E20620CC08E3221F426FD6BC1C0
:1048F000206406C08C3611F4206802C0883641F46A
:10490000F60193FD859193FF81916F018111C1CFD4
:10491000982F9F7D9554933028F40C5F1F4FFFE331
:10492000F9830DC0833631F0833771F0833509F098
:104930005BC022C0F801808189830E5F1F4F442431
:104940004394512C540115C03801F2E06F0E711CD4
:10495000F801A080B18026FF03C0652D70E002C081
:104960006FEF7FEFC5012C870E943D262C0183014C
:104970002C852F77222E17C03801F2E06F0E711CA4
:10498000F801A080B18026FF03C0652D70E002C051
:104990006FEF7FEFC5012C870E9432262C012C85FA
:1049A0002068222E830123FC1BC0832D90E0481633
:1049B0005906B0F4B70180E290E00E94BD233A941A
:1049C000F4CFF50127FC859127FE81915F01B701A6
:1049D00090E00E94BD2331103A94F1E04F1A510843
:1049E0004114510471F7E5C0843611F0893639F568
:1049F000F80127FF07C060817181828193810C5F7C
:104A00001F4F08C060817181882777FD8095982F9E
:104A10000E5F1F4F2F76722E97FF09C090958095DD
:104A2000709561957F4F8F4F9F4F2068722E2AE0BF
:104A300030E0A4010E944826A82EA81844C085375B
:104A400029F42F7EB22E2AE030E025C0F22FF97F24
:104A5000BF2E8F36C1F018F4883579F0B4C0803796
:104A600019F0883721F0AFC02F2F2061B22EB4FE8D
:104A70000DC08B2D8460B82E09C024FF0AC09F2F63
:104A80009660B92E06C028E030E005C020E130E095
:104A900002C020E132E0F801B7FE07C060817181F9
:104AA000828193810C5F1F4F06C06081718180E01D
:104AB00090E00E5F1F4FA4010E944826A82EA81860
:104AC000FB2DFF777F2E76FE0BC0372D3E7FA51482
:104AD00050F474FE0AC072FC08C0372D3E7E05C03B
:104AE000BA2C372D03C0BA2C01C0B52C34FF0DC031
:104AF000FE01EA0DF11D8081803311F4397E09C079
:104B000032FF06C0B394B39404C0832F867809F0B3
:104B1000B39433FD13C030FF06C05A2CB31418F4FD
:104B2000530C5B18B32CB31468F4B70180E290E027
:104B30003C870E94BD23B3943C85F5CFB31410F499
:104B40003B1801C0312C34FF12C0B70180E390E064
:104B50003C870E94BD233C8532FF17C031FD03C056
:104B600088E790E002C088E590E0B7010CC0832F91
:104B7000867859F031FF02C08BE201C080E237FD38
:104B80008DE2B70190E00E94BD23A51438F4B7016F
:104B900080E390E00E94BD235A94F7CFAA94F401D9
:104BA000EA0DF11D8081B70190E00E94BD23A110A4
:104BB000F5CF332009F451CEB70180E290E00E9496
:104BC000BD233A94F6CFF7018681978102C08FEF1B
:104BD0009FEF2C96E2E10C94CA26DC01CB01FC018C
:104BE000F999FECF06C0F2BDE1BDF89A319600B446
:104BF0000D9241505040B8F70895F999FECF92BDFB
:104C000081BDF89A992780B50895A8E1B0E042E007
:104C100050E00C94EF25DC01A40FB51F415050402B
:104C200048F0CB01840F951F2E910E941C26415005
:104C30005040D0F70895262FF999FECF92BD81BD3F
:104C4000F89A019700B4021631F020BD0FB6F8941F
:104C5000FA9AF99A0FBE08950196272F0E941C26F2
:104C60000C941B26FC010590615070400110D8F790
:104C7000809590958E0F9F1F0895FC0161507040A4
:104C800001900110D8F7809590958E0F9F1F089581
:104C9000FA01AA27283051F1203181F1E8946F936D
:104CA0006E7F6E5F7F4F8F4F9F4FAF4FB1E03ED013
:104CB000B4E03CD0670F781F891F9A1FA11D680FB1
:104CC000791F8A1F911DA11D6A0F711D811D911DE4
:104CD000A11D20D009F468943F912AE0269F112459
:104CE0003019305D3193DEF6CF010895462F4770BD
:104CF000405D4193B3E00FD0C9F7F6CF462F4F7018
:104D0000405D4A3318F0495D31FD4052419302D075
:104D1000A9F7EACFB4E0A69597958795779567951B
:104D2000BA95C9F700976105710508959B01AC011B
:104D30000A2E06945795479537952795BA95C9F742
:104D4000620F731F841F951FA01D0895B7FF0C9459
:104D50004B210E944B21821B930B08952F923F926F
:104D60004F925F926F927F928F929F92AF92BF927B
:104D7000CF92DF92EF92FF920F931F93CF93DF9327
:104D8000CDB7DEB7CA1BDB0B0FB6F894DEBF0FBE84
:104D9000CDBF09942A88398848885F846E847D84D1
:104DA0008C849B84AA84B984C884DF80EE80FD80D3
:104DB0000C811B81AA81B981CE0FD11D0FB6F89449
:0E4DC000DEBF0FBECDBFED010895F894FFCF0A
:104DCE003FC8000000320000005E010000FEFFFF41
:104DDE000A0A0A0A6E2F02005749444532000100A2
:104DEE0057494445310041505A4D444D4E4F434171
:104DFE004C4C0101010101010000C206200001001E
:024E0E000000A2
:00000001FF
